:100000000C9434000C9449000C9449000C94490061
:100010000C9449000C9449000C9449000C9449003C
:100020000C9449000C9449000C9449000C9449002C
:100030000C9449000C9449000C9449000C9449001C
:100040000C9449000C9449000C9449000C9449000C
:100050000C9449000C9449000C9449000C944900FC
:100060000C9449000C94490011241FBECFEFD8E036
:10007000DEBFCDBF11E0A0E0B1E0E8E9F9E002C0E9
:1000800005900D92A230B107D9F70E946C000C9434
:10009000CA040C94000081E08093C50083E0809343
:1000A000C400E0ECF0E080818260808386E0809391
:1000B000C20088E98093C10008958FEF87B988B1A5
:1000C000809588B92FEF88E09DE3215080409040D3
:1000D000E1F700C00000F3CF81E087B988B90000E4
:1000E0000000000000000000000018B80000000040
:1000F0000000000000000000000000000000000000
:100100000000000000000000000088B900000000AE
:10011000000000000000000018B80000000000000F
:1001200000000000000000000000000000000000CF
:10013000000000000000000088B90000000000007E
:1001400000000000000018B80000000000000000DF
:10015000000000000000000000000000000000009F
:1001600000000000000088B900000000000000004E
:100170000000000018B800000000000000000000AF
:10018000000000000000000000000000000000006F
:100190000000000088B9000000000000000000001E
:1001A000000018B80000000000000000000000007F
:1001B000000000000000000000000000000000003F
:1001C000000088B9000000000000000000000000EE
:1001D00018B800000000000000000000000000004F
:1001E000000000000000000000000000000000000F
:1001F00088B900000000000000000000000018B8EE
:1002000000000000000000000000000000000000EE
:10021000000000000000000000000000000088B99D
:1002200000000000000000000000000000000000CE
:1002300000000000000000000000000018B80000EE
:10024000000000000000000000000000000088B96D
:1002500000000000000000000000000018B80000CE
:10026000000000000000000000000000000000008E
:1002700000000000000000000000000088B900003D
:100280000000000000000000000018B8000000009E
:10029000000000000000000000000000000000005E
:1002A0000000000000000000000088B9000000000D
:1002B000000000000000000018B80000000000006E
:1002C000000000000000000000000000000000002E
:1002D000000000000000000088B9000000000000DD
:1002E00000000000000018B800000000000000003E
:1002F00000000000000000000000000000000000FE
:1003000000000000000088B90000000000000000AC
:100310000000000018B8000000000000000000000D
:1003200000000000000000000000000000000000CD
:100330000000000088B9000000000000000000007C
:10034000000018B8000000000000000000000000DD
:10035000000000000000000000000000000000009D
:10036000000088B90000000000000000000000004C
:1003700018B80000000000000000000000000000AD
:10038000000000000000000000000000000000006D
:1003900088B900000000000000000000000018B84C
:1003A000000000000000000000000000000000004D
:1003B000000000000000000000000000000088B9FC
:1003C00000000000000000000000000018B800005D
:1003D000000000000000000000000000000000001D
:1003E00000000000000000000000000088B90000CC
:1003F0000000000000000000000018B8000000002D
:1004000000000000000000000000000000000000EC
:100410000000000000000000000088B9000000009B
:10042000000000000000000018B8000000000000FC
:1004300000000000000000000000000000000000BC
:10044000000000000000000088B90000000000006B
:1004500000000000000018B80000000000000000CC
:10046000000000000000000000000000000000008C
:1004700000000000000088B900000000000000003B
:100480000000000018B8000000000000000000009C
:10049000000000000000000000000000000000005C
:1004A0000000000088B9000000000000000000000B
:1004B000000018B80000000000000000000000006C
:1004C000000000000000000000000000000000002C
:1004D000000088B9000000000000000000000000DB
:1004E00018B800000000000000000000000000003C
:1004F00000000000000000000000000000000000FC
:1005000088B900000000000000000000000018B8DA
:1005100000000000000000000000000000000000DB
:10052000000000000000000000000000000088B98A
:1005300000000000000000000000000018B80000EB
:1005400000000000000000000000000000000000AB
:1005500000000000000000000000000088B900005A
:100560000000000000000000000018B800000000BB
:10057000000000000000000000000000000000007B
:100580000000000000000000000088B9000000002A
:10059000000000000000000018B80000000000008B
:1005A000000000000000000000000000000000004B
:1005B000000000000000000088B9000000000000FA
:1005C00000000000000018B800000000000000005B
:1005D000000000000000000000000000000000001B
:1005E00000000000000088B90000000000000000CA
:1005F0000000000018B8000000000000000000002B
:1006000000000000000000000000000000000000EA
:100610000000000088B90000000000000000000099
:10062000000018B8000000000000000000000000FA
:1006300000000000000000000000000000000000BA
:10064000000088B900000000000000000000000069
:1006500018B80000000000000000000000000000CA
:10066000000000000000000000000000000000008A
:1006700088B900000000000000000000000018B869
:10068000000000000000000000000000000000006A
:10069000000000000000000000000000000088B919
:1006A00000000000000000000000000018B800007A
:1006B000000000000000000000000000000000003A
:1006C00000000000000000000000000088B90000E9
:1006D0000000000000000000000018B8000000004A
:1006E000000000000000000000000000000000000A
:1006F0000000000000000000000088B900000000B9
:10070000000000000000000018B800000000000019
:1007100000000000000000000000000000000000D9
:10072000000000000000000088B900000000000088
:1007300000000000000018B80000000000000000E9
:1007400000000000000000000000000000000000A9
:1007500000000000000088B9000000000000000058
:100760000000000018B800000000000000000000B9
:100770000000000000000000000000000000000079
:100780000000000088B90000000000000000000028
:10079000000018B800000000000000000000000089
:1007A0000000000000000000000000000000000049
:1007B000000088B9000000000000000000000000F8
:1007C00018B8000000000000000000000000000059
:1007D0000000000000000000000000000000000019
:1007E00088B900000000000000000000000018B8F8
:1007F00000000000000000000000000000000000F9
:10080000000000000000000000000000000088B9A7
:1008100000000000000000000000000018B8000008
:1008200000000000000000000000000000000000C8
:1008300000000000000000000000000088B9000077
:100840000000000000000000000018B800000000D8
:100850000000000000000000000000000000000098
:100860000000000000000000000088B90000000047
:10087000000000000000000018B8000000000000A8
:100880000000000000000000000000000000000068
:10089000000000000000000088B900000000000017
:1008A00000000000000018B8000000000000000078
:1008B0000000000000000000000000000000000038
:1008C00000000000000088B90000000000000000E7
:1008D0000000000018B80000000000000000000048
:1008E0000000000000000000000000000000000008
:1008F0000000000088B900000000000000000000B7
:10090000000018B800000000000000000000000017
:1009100000000000000000000000000000000000D7
:10092000000088B900000000000000000000000086
:1009300018B80000000000000000000000000000E7
:1009400000000000000000000000000000000000A7
:1009500088B900000000000000000000000018B886
:100960000000000000000000000000000000000087
:1009700000000000000000000000000000002FE761
:1009800034E89EE1215030409040E1F700C0000083
:080990000C946E00F894FFCFF7
:0209980020003D
:00000001FF
